:020000040000FA
:02000000AA292B
:08000800042807200034640005
:10001000061A1128A4190F28201420151128A0143D
:100020002011861A1A28A41D1828201420151A2811
:10003000A01420110800A01F06143B2006104F201A
:100040002010A0160034A01F06140330A7003B2088
:10005000A70B272806104F20A010A0120034A01FC5
:1000600006147D30A7003B20A70B332806104F2035
:1000700000340A303C282308A1007430402878302E
:10008000A2004228A20B4128241806157830A200AD
:100090004928A20B48280611A10B3F28072823084E
:1000A000A1007830A2005428552856280000A20B41
:1000B0005328A10B512807280520A41FCF28201C56
:1000C000A018CF286620CF28063067280230A70066
:1000D0004F20A70B68280034A8002808A807031D94
:1000E000732866200034031877281B206D282320EE
:1000F0006D28A50000308A0025088207FC347C3476
:100100003C341C340C3404348434C434E434F434C7
:100110000315492A0315D02A0315172A03158C2A1B
:100120000315202B0315FC2A7830A100F030A20023
:1001300005209A28A20B9828A10B9628A01C20180D
:10014000A3282A10A4282A1400342016A017241447
:1001500050306C206400861FAA288E208A2003114C
:10016000A50000308A00250882074429492946292C
:100170005529202906294F2942298E2993293D29CD
:1001800027080319C528A703CA288611F03083164B
:100190008600831264002410A4182414A0010520F2
:1001A000241FD528A0181829F028061E861ADC2836
:1001B0002017A01AEC28EE28201FE3282013A41EE5
:1001C000D928A0015C282018A01CE8282019EC28B8
:1001D0002018EE28A01CF02823205C281B205C2877
:1001E000861FF628630000000B10C028F830831625
:1001F000860083129420861B00299420861FA52840
:10020000003088202F200630A700C028A41C24100E
:1002100006143920A0180E29201C09291930A8001D
:100220006400061A861E0E29A80B10290610C02885
:10023000A41C24100614A0103920A0181B290E2974
:10024000AB0140306C208E208030290203193D29FB
:100250002B182F2990200311AA002B14212992205A
:100260000311AA07031C3D29FB302A07031C3D2963
:10027000A6008C200311A3008B2932308C2950302A
:100280006C200E2908304729023047294030A40647
:100290003F292030A4066030A41E88308C2980308D
:1002A000A4066030A41FA0308C292D3084004F306C
:1002B000AA0040306C208E205630290203196D2987
:1002C00080302902031D6629023067292908800031
:1002D000840A00308000AA0B59295030A700A703D8
:1002E00027082D3E840000088316031364009C1821
:1002F00076299A0083122708831603139B009C1308
:100300001C1555309D00AA309D009C141C118312B1
:10031000A708031D6F2950306C20C02800308820AA
:100320000630A700C02805302607AB01AA000A3016
:10033000AA02031C9D29AB0A9829AA072B080319B6
:10034000A429792003116C202A08792003116C203C
:1003500008308F29F83083168600003085000E3073
:1003600081008312860108308B00031AB92970308E
:100370008C290530A6008C200311A300B330A40003
:100380005030A7006400A7032708831603139B00BF
:100390001C141A088312A80027082D3E8400280880
:1003A0008000A708031DC229831664001C18D529E4
:0C03B0008312A0175030861E88308C2964
:100400008000840A00342C08AC0AA50002308A005F
:10041000250882071834183418348C340234033415
:1004200002340034023470346834E0340034A500FF
:1004300002308A0025088207D434B03497348434DB
:1004400075346A346034583451344B344634423451
:100450003E343A3437343534323430342E342C345C
:100460002A342834273425342434233422342134C4
:1004700020341F341E341D341C341B341B341A34F6
:100480001934193418341834173417341634163410
:100490001534AC00A0194E2A0322502A0008840A01
:1004A000A80000302802031D5C2AA01D592AA011B3
:1004B0004A2A0311A01100340330280203196C2AC0
:1004C0000130280203194A2A02302802031D702A2B
:1004D0000311642003154A2A2D308400A0154A2AEE
:1004E000861E742A061A7A2A6400A001861A061E3D
:1004F000742A592A2808A807031D822A0311662096
:1005000003154A2A0318882A03111B200315702A91
:10051000031123200315702AA9010830A800DC303C
:10052000A200AA30A1000330AC000311052003157E
:10053000201C9C2AA018AB2A2018B12AA018B62A81
:10054000A20B952ADC30A200A10B952AAA30A100AB
:10055000AC0B952AC52AA41EAF2AFC30A005A01A10
:10056000B62A03111B2003150310BA2A03112320F6
:1005700003150314A90DA80BBE2ACD2ADC30A20056
:10058000AA30A1000130AC00952A0314C82A031038
:10059000A90DA80BC72A031100348030A900CB2A6B
:1005A0002908A800603028020319003420302802EE
:1005B00003190134B03028020319023448302802EC
:1005C000031903341030280203190434C030280200
:1005D00003190534303028020319063498302802F4
:1005E00003190734201290302802031908347030A0
:1005F0002802031909340A347C3029020319813492
:100600003C302902031982341C3029020319833437
:100610000C3029020319843404302902031985346B
:100620008430290203198634C4302902031987341F
:10063000E430290203198834F4302902031989347B
:10064000C030290203198034FC3029020319803498
:100650007C30290203198A343C302902031994346E
:100660001C30290203199E340C3029020319A834C6
:02067000003454
:02400E001C3F55
:10420000A800D800020088006000480020001000CC
:10421000400002003C001C00A800E00002009000EA
:104220004000020028007C00680090009800020016
:104230004800F000A80002007800A000FC00E400A4
:10424000980010000200900040006800C400E400E4
:1042500002006000A000C000020090002000680082
:1042600002006800700050000200040070000200AC
:104270000200A800D800020088006000480020006A
:104280001000400002003C001C00A800E0000200FA
:1042900090004000020028007C0068009000980018
:1042A00002004800F000A80002007800A000FC0016
:1042B000E400980010000200900040006800C40074
:1042C000E40002006000A000C00002009000200096
:1042D00068000200680070005000020004007000D6
:0242E0000000DC
:00000001FF
